:02000000F728DF
:0800080069288C0081018316B8
:10001000C030810508008C0081018316C030810545
:100020000130810483120B110B1D14288C0B132833
:1000300008009A00861008308C002A201A188614AE
:100040001A1C86109A0C2A208C0B1E2886142A2033
:100050002A2008001D308D0030280B308D003028FC
:100060008D0B302808002D200618452808308C00FC
:100070002A2006189B17061C9B130C0B9B0C8C0B41
:1000800038282A20061C9B0108009B01EE289500B9
:1000900008309400951F0511951B0515950D00005E
:1000A000851500001510051A15148511940B4A28A2
:1000B00008001908840017088000840A18088000C6
:1000C000840A04089900283C031D08002030990088
:1000D00008008B138B1B69289C00030E9D00830175
:1000E0000A089E008A01831304089F000D3019201E
:1000F0000A3019200A3019205030192052301920A6
:100100004530192043301920493019205330192027
:10011000493019204F3019204E3019202030192035
:10012000443019204930192047301920493019200E
:1001300054301920413019204C301920203019201A
:10014000413019204C3019205430192049301920E1
:100150004D301920453019205430192045301920D0
:10016000523019200D3019200A3019203130192051
:100170003930192039301920393019202D30192003
:100180003230192030301920303019203130192008
:1001900020301920623019207930192020301920A0
:1001A000503019206530192074301920653019201D
:1001B00072301920203019204C3019207530192048
:1001C00065301920743019206830192069301920E1
:1001D0000D3019200A3019200A3019201F08840018
:1001E0001E088A001D0E83009C0E1C0E090083163B
:1001F0008610061401138312861490308B04831624
:10020000F03085008312033085006620FC308505C0
:10021000343047200330850401300B20FC30850545
:10022000F83047200330850401300B20FC30850571
:10023000203047200330850403300B20FC30850537
:10024000243047200330850401300B20FC30850525
:100250008430472085140030472003308504103057
:1002600096009701980101300B20FC308505843001
:10027000472015088E0085140030472015088F0090
:10028000033085040F0897070318980A0E0898078B
:10029000960B3329F0309705970E980E18059704A2
:1002A0000F309805592097019801203084000008EC
:1002B00097070318980A840A00089807840A040814
:1002C000283C031D5729970C970C1713181817175C
:1002D000971398189717980C980C181398131708D9
:1002E000910018089000FC308505C4304720851423
:1002F00000304720033085041030960097019801A4
:1003000001300B20FC308505C430472015088E00D5
:1003100085140030472015088F00033085040F082E
:1003200097070318980A0E089807960B8029F03053
:100330009705970E980E180597040F309805170823
:1003400093001808920054301920553019201008D5
:1003500019201108192012081920130819202F300C
:0803600019203F301920262965
:02400E00F13F80
:00000001FF
